:020000040000fa
:08000000a2060400000000004c
:020000040000fa
:020000040002f8
:04afe000dfff00008f
:020000040000fa
:020000040002f8
:04afe400ffff00006b
:020000040000fa
:020000040002f8
:04afe80078ff0000ee
:020000040000fa
:020000040002f8
:04afec007dff0000e5
:020000040000fa
:020000040002f8
:04aff00078ff0000e6
:020000040000fa
:1000080000000000000000000000000000000000e8
:100018009a06000000000000000000000000000038
:100028000000000000000000000000000e090000b1
:1000380000000000000000000000000000000000b8
:100048004e0900000000000000000000d809000070
:10005800440a0000700a00000000000000000000d0
:100068000000000000000000000000000000000088
:100078000000000000000000000000000000000078
:100088000000000000000000000000007a090000e5
:10009800a8090000000000000000000000000000a7
:1000a8000000000000000000000000000000000048
:1000b8000000000000000000000000000000000038
:1000c8000000000000000000000000000000000028
:1000d8000000000000000000000000000000000018
:1000e8000000000000000000000000000000000008
:1000f80000000000000000000000000000000000f8
:1001080000000000000000000000000000000000e7
:1001180000000000000000000000000000000000d7
:1001280000000000100a00000000000000000000ad
:1001380000000000000000000000000000000000b7
:1001480000000000000000000000000000000000a7
:100158000000000000000000000000000000000097
:100168000000000000000000000000000000000087
:100178000000000000000000000000000000000077
:100188000000000000000000000000000000000067
:100198000000000000000000a20a0000ce0a0000d3
:1001a800fa0a000000000000000000000000000043
:1001b8000000000000000000000000000000000037
:1001c8000000000000000000000000000000000027
:1001d8000000000000000000000000000000000017
:1001e8000000000000000000000000000000000007
:1001f80000000000000000000000000000000000f7
:1002080000000000000000000000000000000000e6
:1002180000000000000000000000000000000000d6
:1002280000000000000000000000000000000000c6
:1002380000000000000000000000000000000000b6
:1002480000000000000000000000000000000000a6
:100258000000000000000000000000000000000096
:100268000000000000000000000000000000000086
:0c0278000000000000000000000000007a
:020000040000fa
:10040000803e2000030007008100e900fcff3a0065
:1004100000000600831f7800c20320000400bc0017
:1004200066015100e0815900f23fb1000380b10044
:1004300006003500ee03090000000000423fb10055
:100440000380b100fbff3d001200b000223fb0006e
:10045000020035000280090000000000cf01780092
:10046000000006000001eb00869fbe00889fbe00d2
:100470008a9fbe008c9fbe00820578000004be00eb
:10048000e00107000800be006420e1000700390019
:1004900002003a00f1ff2f00f0ff27000160a000ea
:1004a0001202200012918800560037006120e100fe
:1004b00003003a000b00a70001f8230051003700a9
:1004c00001f0a10002002100936424005200070003
:1004d0000800be0005003500b2fd2000930c24008a
:1004e00004002000690007000004be000005eb00c6
:1004f0000b00a6004f0dde0001f0a1000004be00bd
:1005000032982f0023ea23000f0107000001eb00bf
:10051000030020000b00a70003f82300ac00070035
:100520003e0107000000a7000a00a20080010700aa
:100530000b00e000030032000200200003f0230063
:10054000a200070001f0a2000006be000200200089
:1005500093042400fc0007000801be009c00070073
:10056000809fbe000c00be0022a22a00d3a7230059
:10057000f50007004f01be00950007000004be0013
:1005800001f0a100020020000398230022000700d0
:100590000800be00190035000001be00ea00070097
:1005a0000006be00b2c52900e3622300e600070092
:1005b00022222b00f3942b00850007000c01be00c3
:1005c000e1000700e273280083c0230080000700d9
:1005d0000c01be00dc00070042aa2a00a3e22b00a7
:1005e0007b0007000c01be00d70007000801be0019
:1005f000d50007000801be00750007000a00a7002b
:1006000001f0a2004f06be004f05be004f04be0021
:100610004f03be000000060014002000889fbe00ab
:100620008a9fbe00841f78006e0107004f0078008b
:1006300011003300f0ff2f00838f6c0006003b0099
:10064000040565000a00a7000800370009f0a600ad
:100650001000200008003700820f5400838f5c00d8
:10066000030039001000200001003e0000002000bf
:1006700009f0a7000000ea004f05be004f04be00cd
:100680000000e0000000060014002000869fbe006d
:10069000889fbe008a9fbe008c9fbe004f26dd0053
:1006a00050010700920133006120e1004300320055
:1006b0006250e10041003e003e0039006420e1004c
:1006c0003c003200058255000f003b000402e800a8
:1006d00038003a00800f5300818f5b0035003400f2
:1006e0000800be0003f0a10001f0a60003f0a00086
:1006f0000cf0a70036000700860137000603430010
:1007000087834b000c4646000005530081855b0043
:10071000020033000a03be000c00a0000402e9003e
:10072000f6ff3b00850578000602430087824b00f8
:1007300004003a006000b80009f0a70001f0a00032
:10074000740137000002520081825a000704e00061
:10075000040033000603430087834b008b05e90048
:10076000faff3700090578000604be000203be0048
:100770006011b80038010700e00f5200e08f5a0006
:100780000700350002003c000c08a3000400320002
:100790000601be0003f0a0000cf0a7000c0007004b
:1007a0000a85680001f0a1000af0a70001f0a0008e
:1007b000580137000800be00560137001002200023
:1007c0000cf0a600109188005701370003f0a2003a
:1007d000869fbe00889fbe008a9fbe008c9fbe0081
:1007e00000010700420133006450e1004f00320075
:1007f0006420e1005200320003826c0007003b00dd
:100800000905d0000306d000820f54000c065d00dd
:1008100002003900020032008901780003067800e6
:100820008582550004003d000003fd008103fd00aa
:100830008502ea008b854200840f720002003b00b3
:1008400060001000e08018006011b8000005eb00a7
:100850007a28e1000a00390006007800c75ddd0053
:10086000f707b200878075002d0037008281710084
:100870000a017800610560008180d1000080d3000a
:100880008502e900f9ff3b00060440008784480028
:1008900002003b0060041400e0841c000988a300ef
:1008a000070032008a817100828171006101640059
:1008b0008904d1000884d3008b05e80017003700b5
:1008c0000978a30013003a000b00e0001300340085
:1008d0008b05e9000804440089844c000a44740034
:1008e0000978a3000d003a000b00e0000700340077
:1008f0008b05e9000804440089844c0001003a009b
:100900000b0020000978a300f7ff32000001eb0084
:1009100002003700828171000a017800ce000700d2
:100920000cf0a70001f0a000fa0037006420e100fd
:1009300002003a00838f6c00fb0033000801be0008
:100940000200be00f3003700869fbe00889fbe00f5
:100950008a9fbe008c9fbe00a2000700e400330007
:1009600003866c006450e100240032006420e10042
:10097000270032006150e100220032006120e100d6
:10098000210032008b854200eb07b1000134b80032
:10099000003ab8000804420089844a00013ab800cd
:1009a0000030b8008880400009014a00040033008c
:1009b0000000400081804800020149008b05e900e9
:1009c000c909dd008301700001003200130020001e
:1009d000c814de004814dd004709de001200b20032
:1009e000c808de00088470009b00070001f0a10029
:1009f0000cf0a70001f0a000c60037006120e10064
:100a0000c90032000801be000200be00f7ff370037
:100a10006150e100fcff3a00c3003700829fbe0036
:100a20000001be00770007000470a70003f0a100da
:100a30006509b100180032000e0035006828e10099
:100a400007003500f0ff2f00f1ff27000300e00052
:100a500015003b00010028004f01be00000005000a
:100a600000004000818048008502e900fcff3a0058
:100a700009003700f88f420003003c008000eb00c3
:100a80004f01be00000005008100d1000080d300ae
:100a90008502e800fcff3a000300e00002003b0092
:100aa00060001000e08018004f01be00000006004a
:100ab000829fbe000001be00520007000470a70024
:100ac00003f0a10003f8a30015003a006509b10086
:100ad000110032000a0035006928e10003003500ea
:100ae000010028004f01be0000000500000040008a
:100af000818048008502e900fcff3a0006003700cb
:100b0000f88f4200060035008100d1000080d3003c
:100b10008502e800fcff3a004f01be00000006001d
:100b20008000eb004f01be00000005008000eb00dc
:100b3000829fbe00889fbe008a9fbe00010578008c
:100b40000100e0000400350008003c000000e00067
:100b5000200032000500370060001000e08018001f
:100b600002003b0001f024001a0037000004be0020
:100b70006011b8006b0920000982cf000200390023
:100b80000882cf000441b000694252000e003200da
:100b900008003b0082817100610164008904d1007a
:100ba0000884d3008b05e8000442e800f9ff3a000e
:100bb000050037000804440089844c008b05e900d7
:100bc0000442e900fbff3a00230007000af0a700f7
:100bd00001f0a0004f05be004f04be004f01be0053
:100be000000006000004be00060007000003be006f
:100bf0000405be000200be0002000700844f75001d
:100c000000000600c70ade00f107b200f50fb200cf
:100c100008003200e1cf4200020032000170a00063
:100c200024000500810f7000010032000408050057
:100c300044000500810f700002003a001400050016
:100c40008502e9000000400081c04800fcff3b0035
:100c50000170a00024000500810020006180550083
:100c60000b003d000b00200061fe2f000100e100a1
:100c70001d00340082817100610164008904d1008b
:100c80000884d3000000e800faff3a007100200059
:100c9000610064000300700002006000090032007f
:100ca00061044400e0844c000988a500050032007e
:100cb0008b05e8006808e10002003a008904d100d1
:100cc0000884d300f20f20000258e10005003d0027
:100cd000c75ddd00f907b200898075000800780063
:100ce000000006000bf827008b00780000000500cc
:100cf0000200be006450e100050036006420e100ff
:100d0000020036000968a30001003a000800be0096
:100d10000160a0004f06be004f05be004f04be009c
:100d20004f03be0000000600f0ff2f00f1ff270078
:100d3000f8ff37000020ef000220ef00c088a90074
:100d4000004006000f002100b02e210000018800a5
:100d5000000000000000eb00000778000c00090014
:100d6000002f78000007eb005420ef000e2eef005c
:100d70001e2eef000000eb00a1212100e51d09005f
:100d80008018780040a7a900a10020009cfd070062
:100d9000e0022000303a880044e7a90044c7a900d7
:100da0004407a9004427a9004447a9004467a900b3
:100db0004487a900300020000600fc0031742000a8
:100dc00082072000a3092000824878008348780029
:100dd00080487800113a8000618070000600fc00b5
:100de00021742000620420007305200082487800ee
:100df00083487800804878004427ef00e002200014
:100e0000303a8800300020000d00fc0031742000d2
:100e100082072000a30920008248780083487800d8
:100e20008048780000002000217420006204200027
:100e30007305200082487800834878008048780055
:100e400042a7ae00feff3700813e20006cfd070088
:100e500010c0b30086e6b70090c2b300c4e6b70086
:100e60001002200000708800007825008070880043
:100e700010aea90010cea900102ea900002ea900c6
:100e8000100ea900570507003d0607005d07070083
:100e90003b0707000000eb0081772100ff000900fd
:100ea000805878005272ef005372ef003e32ef002c
:100eb0004032ef000080eb000177210003000900c1
:100ec000801878002a32ef0010cea90014cea900b5
:100ed0006e32a9003432ef004188a80041a8a90071
:100ee00041c8a80000a1ef0080938000100888008e
:100ef00080938000d091880004a1a8000481a900fb
:100f000005e1a8000068a9002068a8001061a800f9
:100f10001021a90011e1a80011a1a90010a1a800a9
:100f20001081a8000621ef000a21ef000ca1ef00bc
:100f30000ea1ef004408a9004428a9004448a900d4
:100f40000108a9002108a80021e1a80021a1a90009
:100f500020c1a90020a1a8002081a8002021a9006b
:100f60004e08a8004e28a9004e48a8000388a900f2
:100f700040922000e00888002388a8002002a900f1
:100f80002022a9002042a90020a2a9002062a900d5
:100f90002082a90020e2a9002102a9002122a900a3
:100fa000700720004011880022a2a90022c2a900d7
:100fb00022e2a90021e2a8002182a9004588a90017
:100fc00045a8a80045c8a8002168a8002828a800ae
:100fd0000e0ea80021e3a9002143a80021a3a90027
:100fe0002123a9002103a90020e3a80020c3a80011
:100ff00020a3a8002083a9002043a90023e3a9007f
:1010000023c3a90023a3a9002343a9002323a900e4
:101010002303a90022c3a90022a3a9002283a900b7
:101020002263a9002243a9002223a9002203a900c8
:101030002563ef0024e3ef003223ef002823ef00c5
:101040002623ef002e23ef003023ef0021a8a80075
:1010500001a8a90021e3a8002bc8a9002be8a9003a
:101060002c08a9000bc8a9000be8a9000c08a900ce
:1010700001eca90001aca900016ca900014ca90078
:10108000012ca900010ca90000eca900008ca9000a
:1010900000aca90000cca900000ca900002ca900fc
:1010a000004ca900006ca900202cef00402cef00a0
:1010b000602cef0004acef00020ca900022ca90088
:1010c000024ca900000028003061880000002800c0
:1010d000306288000000280030638800282cef0070
:1010e000482cef00682cef000aacef0023eca800be
:1010f00023cca80023aca900238ca900236ca90051
:10110000234ca800232ca900230ca900222ca90001
:1011100043eca80043cca80043aca900438ca90031
:10112000436ca900434ca800432ca900430ca90020
:1011300063eca80063cca80063aca900638ca80092
:10114000636ca900634ca800dabc2a001b3224009f
:1011500030002c00fa608800fb6088002061880065
:10116000dabc2a001b32240000402c00fa60880000
:10117000fb60880010618800dabc2a001b32240062
:1011800030002c00fa608800fb6088002062880034
:10119000dabc2a001b32240000402c00fa608800d0
:1011a000fb60880010628800dabc2a001b32240031
:1011b00030002c00fa608800fb6088002063880003
:1011c000dabc2a001b32240000402c00fa608800a0
:1011d000fb60880010638800218ca900418ca90065
:1011e000618ca900216ca900416ca900616ca90067
:1011f000214ca900414ca900614ca90020eca80099
:1012000040eca80060eca8003e2cef005e2cef0044
:101210007e2cef0001eca80018013700ff3ffc0016
:101220004200f8003600f8004400f8008e1f7800f5
:101230000e0020000d000900be1f78003200f800eb
:101240000100fc000068a9000021ef00d09180009f
:1012500010088800609180003061880070918000e3
:101260003062880080918000306388006572ec00f5
:10127000ff3ffc003200f900ae0120000d00090024
:101280004f1778004f0778004400f9003600f90046
:101290004200f9000100fc0000400600ff3ffc0096
:1012a0004200f8003600f8004400f8008e1f780075
:1012b0000e0020000d000900be1f78003200f8006b
:1012c0000100fc000108a900ff3ffc003200f9000a
:1012d000ae0120000d0009004f1778004f0778007d
:1012e0004400f9003600f9004200f9000100fc005a
:1012f00000400600ff3ffc004200f8003600f80006
:101300004400f8008e1f78000e0020000d00090038
:10131000be1f78003200f8000100fc000368a9003d
:101320001421ef00ff3ffc003200f900ae01200065
:101330000d0009004f1778004f0778004400f900ae
:101340003600f9004200f9000100fc0000400600f0
:10135000ff3ffc004200f8003600f8004400f800af
:101360008e1f78000e0020000d000900be1f7800bf
:101370003200f8000100fc000388a9001821ef00ea
:101380002023a800ff3ffc003200f900ae0120003e
:101390000d0009004f1778004f0778004400f9004e
:1013a0003600f9004200f9000100fc000040060090
:1013b000ff3ffc004200f8003600f8004400f8004f
:1013c0008e1f78000e0020000d000900be1f78005f
:1013d0003200f8000100fc000168a9005272ec0024
:1013e00052d2bf008080fb00301180008277210044
:1013f00080707900ff3ffc003200f900ae01200050
:101400000d0009004f1778004f0778004400f900dd
:101410003600f9004200f9000100fc00004006001f
:10142000ff3ffc004200f8003600f8004400f800de
:101430008e1f78000e0020000d000900be1f7800ee
:101440003200f8000100fc000828a9002242ae008a
:10145000000037002222af002222a900ff3ffc003b
:101460003200f900ae0120000d0009004f1778008e
:101470004f0778004400f9003600f9004200f900f7
:101480000100fc0000400600ff3ffc004200f800a5
:101490003600f8004400f8008e1f78000e0020008f
:1014a0000d000900be1f78003200f8000100fc00aa
:1014b0000188a900ff3ffc003200f900ae012000c6
:1014c0000d0009004f1778004f0778004400f9001d
:1014d0003600f9004200f9000100fc00004006005f
:1014e000ff3ffc004200f8003600f8004400f8001e
:1014f0008e1f78000e0020000d000900be1f78002e
:101500003200f8000100fc0000188000e091880023
:1015100001a8a9002003a900ff3ffc003200f90048
:10152000ae0120000d0009004f1778004f0778002a
:101530004400f9003600f9004200f9000100fc0007
:1015400000400600ff3ffc004200f8003600f800b3
:101550004400f8008e1f78000e0020000d000900e6
:10156000be1f78003200f8000100fc000bc8a90083
:10157000ff3ffc003200f900ae0120000d00090021
:101580004f1778004f0778004400f9003600f90043
:101590004200f9000100fc0000400600ff3ffc0093
:1015a0004200f8003600f8004400f8008e1f780072
:1015b0000e0020000d000900be1f78003200f80068
:1015c0000100fc000be8a900ff3ffc003200f9001d
:1015d000ae0120000d0009004f1778004f0778007a
:1015e0004400f9003600f9004200f9000100fc0057
:1015f00000400600ff3ffc004200f8003600f80003
:101600004400f8008e1f78000e0020000d00090035
:10161000be1f78003200f8000100fc000c08a90091
:10162000ff3ffc003200f900ae0120000d00090070
:101630004f1778004f0778004400f9003600f90092
:101640004200f9000100fc000040060053d2bf0038
:101650005252e300070032005372ec0053d2bf0035
:101660000080fb008177210060c0780054f2b70051
:101670000100370054f2ef000000060005e1a80069
:10168000500880000092880030088000f0918800a7
:10169000eeff0700e0ceb3005452b500060039005b
:1016a000e0cfb3005452b50001003900010037000b
:1016b0005572ef006d01370054f2ae00370037006d
:1016c0005572ef00d0c8b3005452e30005003a0051
:1016d00054d2bf0055f2b70056f2ef0057f2ef00b8
:1016e0002d003700d0c9b3005452e30005003a0082
:1016f00054d2bf0055f2b70058f2ef0059f2ef0094
:1017000025003700d0cab3005452e30005003a0068
:1017100054d2bf0055f2b7005af2ef005bf2ef006f
:101720001d003700d0cbb3005452e30005003a004f
:1017300054d2bf0055f2b7005cf2ef005df2ef004b
:1017400015003700d0ccb3005452e30004003a0037
:1017500054d2bf0055f2b7005ef2ef000e00370022
:10176000d0cdb3005452e30004003a0054d2bf007d
:1017700055f2b7005ff2ef0007003700d0ceb3009c
:101780005452e30004003a0054d2bf0055f2b700af
:1017900060f2ef0061f2ef00340137005552e200d1
:1017a00002003a003101370030013700d0c8b300e1
:1017b0005552e30045003a0000e0ef005652e300c6
:1017c00003003a0054d2bf0056f2b7003e00370083
:1017d00054d2bf0057f2b70080c1b3005652e300a5
:1017e00038003a005752e2001b003a0014cea9001c
:1017f0000000280060918800000028007091880097
:1018000000002800809188006b72ef003412a9005c
:101810002a12ae000400370070b7ef0072b7ef0075
:101820006312a8002a12a900140ea9002a32ae00e1
:101830000400370074b7ef0076b7ef006312a8001a
:101840002a32a90080938000c0918800c091800056
:10185000d09188001b003700022eae00190037001f
:101860003412a8000280200057d2bf000080fb0085
:101870000200b8000001be0082bb880093bb880054
:1018800082bb800093bb8000f091800001928000b9
:1018900002004000838048000001be0082bb880037
:1018a00093bb88002a12a8006312a8002a32ae0057
:1018b0000300370074b7ef0076b7ef002a32a900b3
:1018c000140ea90056f2ef00e8003700d0c9b300ab
:1018d0005552e3006f003a0000e0ef005852e30079
:1018e00003003a0054d2bf0058f2b7006800370036
:1018f00054d2bf0059f2b7005952e2001c003a001e
:1019000080c1b3005852e30018003a0014cea90079
:101910000000280060918800000028007091880075
:1019200000002800809188003412a9002a12ae001d
:101930000400370070b7ef0072b7ef006312a80021
:101940002a12a9002a32ae000300370074b7ef0054
:1019500076b7ef002a32a90080938000c0918800fa
:10196000c0918000d0918800140ea9004700370074
:1019700080c1b3005852e30044003a0059d2bf007e
:101980006cf2b700022eae003c0037006cd2bf00f4
:101990000080fb00000040000127210060807800eb
:1019a000c0918800c1918000d0918000808f50004c
:1019b0000d003a006cd2bf000080fb004200de0048
:1019c00001022000008050006bf2b7002a32ae0006
:1019d000040037002a32a90074b7ef0076b7ef0091
:1019e0006312a8001b003700d2918000808721007d
:1019f000604079006df2b700d0918000c191800005
:101a0000808f500009003600401f20000100200098
:101a1000f29180000392800002014000838148001f
:101a2000a2bb8800b3bb8800080037000019200063
:101a300001002000f291800003928000020140002a
:101a400083814800a2bb8800b3bb88002a32a8006b
:101a50006312a8003412a9002a12ae000400370055
:101a600070b7ef0072b7ef006312a8002a12a90046
:101a700014cea800140ea8000400370014cea9004c
:101a8000140ea90000c2b3006bf2b70058f2ef00c9
:101a900076003700d0cab3005552e30045003a0043
:101aa00000e0ef005a52e30003003a0054d2bf00b6
:101ab0005af2b7003e00370054d2bf005bf2b700c5
:101ac00080c1b3005a52e30038003a0012ceae0093
:101ad0003600370010cea90014cea8003412af0093
:101ae000320037005bd2bf000080fb0000004000e6
:101af0000127210060807800c0918800c19180009a
:101b0000d0918000808f50000d003a005bd2bf0062
:101b10000080fb004200de00010220000080500037
:101b20006bf2b7002a32ae00040037002a32a90057
:101b300074b7ef0076b7ef006312a8001b00370000
:101b4000d291800080872100604079006df2b7005b
:101b5000d0918000c1918000808f50000900360034
:101b6000401f200001002000f291800003928000bd
:101b70000201400083814800a2bb8800b3bb8800fb
:101b8000080037000019200001002000f2918000b9
:101b9000039280000201400083814800a2bb8800bc
:101ba000b3bb88002a32a8006312a8005af2ef00e3
:101bb0002e003700d0cbb3005552e3000b003a00a3
:101bc00000e0ef005c52e30003003a0054d2bf0093
:101bd0005cf2b7000400370054d2bf005df2b700da
:101be000c60107005cf2ef0020003700d0ccb30044
:101bf0005552e30007003a0000e0ef005e52e300b8
:101c000003003a0054d2bf005ef2b7005ef2ef006c
:101c100016003700d0cdb3005552e30007003a005c
:101c200000e0ef005f52e30003003a0054d2bf002f
:101c30005ff2b7005ff2ef000c003700d0ceb300c8
:101c40005552e30009003a0000e0ef006052e30063
:101c500003003a0054d2bf0060f2b700030037001f
:101c600054d2bf0061f2b70060f2ef00022eaf0065
:101c70009d003700010020003ff2af001140b0008e
:101c80006e12af001140b100970032006e12a80032
:101c90003ff2ae006e12a900e09180004500de0028
:101ca0006ff2b7006f52e2007e0036006e32af0076
:101cb000410037006fd2bf000080fb0000004000f1
:101cc0000127210060807800c0918800c1918000c8
:101cd000d0918000808f50000d003a006fd2bf007d
:101ce0000080fb004200de00010220000080500066
:101cf0006bf2b7002a32ae00040037002a32a90086
:101d000074b7ef0076b7ef006312a8002100370028
:101d1000d291800080872100604079006df2b70089
:101d20006dd2bf000080fb004200de0001022000f7
:101d3000008050006bf2b700d0918000c19180000c
:101d4000808f500009003600401f20000100200055
:101d5000f2918000039280000201400083814800dc
:101d6000a2bb8800b3bb8800080037000019200020
:101d700001002000f29180000392800002014000e7
:101d800083814800a2bb8800b3bb88002a32a80028
:101d90006312a8003412a9002a12ae000400370012
:101da00070b7ef0072b7ef006312a8002a12a90003
:101db0006e32a800380037006fd2bf000080fb00f1
:101dc000000040000127210060807800c091880059
:101dd000c1918000d0918000808f50000d003a00aa
:101de0006fd2bf000080fb004200de000102200035
:101df000008050006bf2b7002a32ae0004003700ba
:101e00002a32a90074b7ef0076b7ef006312a8007a
:101e100021003700d2918000808721006040790046
:101e20006df2b7006dd2bf000080fb004200de0003
:101e300001022000008050006bf2b700d0918000ba
:101e4000c1918000808f500009003600401f2000a3
:101e500001002000f2918000039280000201400006
:101e600083814800a2bb8800b3bb8800080037000c
:101e70000019200001002000f291800003928000f0
:101e80000201400083814800a2bb8800b3bb8800e8
:101e90002a32a8006312a80014cea800140ea800cd
:101ea0001100370014cea9000000280060918800be
:101eb00000002800709188000000280080918800b0
:101ec0006b72ef003412a9002a12ae000400370032
:101ed00070b7ef0072b7ef006312a8002a12a900d2
:101ee000140ea9006e32a9006312af00e6000700cd
:101ef00020c0b3006252b50062003100f291800050
:101f0000039280003092800041928000800f510047
:101f1000818f59004f00390049f2a8006252e20057
:101f200013003a0014cea900000028006091880038
:101f3000000028007091880000002800809188002f
:101f400000c2b3006bf2b70070b7ef0072b7ef00da
:101f50003412a9002a12a9006e32a90080938000d1
:101f6000c0918800c0918000d0918800380037006f
:101f700010c0b3006252e30035003a00d1918000f6
:101f8000c0918000808f500008003a0074b7ef00c5
:101f900076b7ef002a32a900c29180008087210025
:101fa000604079006df2b70023003700d1918000c6
:101fb000c0918000808f50000e0031003a32ec005a
:101fc000d291800080872100604079006df2b700d7
:101fd000401f200001002000f29180000392800049
:101fe0000201400083814800a2bb8800b3bb880087
:101ff00011003700c0918000d1918000808f500087
:102000000d0036003a32ed000019200001002000da
:10201000f291800003928000020140008381480019
:10202000a2bb8800b3bb8800d291800080872100ca
:10203000604079006df2b7006dd2bf000080fb00f8
:102040004200de0001022000008050006bf2b70069
:102050008d00070041f2ae00090037000621ef00b5
:102060000a21ef003e32ef004032ef000080eb002b
:102070000177210003000900801878007ffd3700f8
:102080000400370041f2ae00020037000621ef00e5
:102090000a21ef0064d2bf006552e30075003200f0
:1020a0002068a9003412af00370037006bd2bf00a0
:1020b0006552b40068f2b70065d2bf000080fb0033
:1020c000000040000137210060807800d090880037
:1020d00068d2bf000080fb000000400001372100f3
:1020e000608078001a12b4006091880065d2bf0049
:1020f0005041b00066f2b7006bd2bf006652b40028
:1021000069f2b70066d2bf000080fb00000040000b
:102110000137210060807800d090880069d2bf002c
:102120000080fb0000004000013721006080780043
:102130001a12b4007091880065d2bf00b042b0009e
:1021400067f2b7006bd2bf006752b4006af2b70003
:1021500067d2bf000080fb00000040000137210073
:1021600060807800d09088006ad2bf000080fb00b9
:102170000000400001372100608078001a12b4008e
:1021800080918800380037002a12ae0030003700f6
:1021900065d2bf000080fb00000040000137210035
:1021a00060807800d090880065d2bf000080fb007e
:1021b0000000400001372100608078001a12b4004e
:1021c0006091880050c1b3006552b50066f2b70057
:1021d00066d2bf000080fb000000400001372100f4
:1021e00060807800d090880066d2bf000080fb003d
:1021f0000000400001372100608078001a12b4000e
:1022000070918800b0c2b3006552b50067f2b700a4
:1022100067d2bf000080fb000000400001372100b2
:1022200060807800d090880067d2bf000080fb00fb
:102230000000400001372100608078000091880094
:10224000d09080002012bc008291880006003700e8
:10225000000028006091880000002800709188002c
:10226000000028008091880065d2bf0064f2b700aa
:102270002068a8004032af0014aea8004032ae0083
:1022800014aea900fefc370062f2ef0049f2a8008c
:102290002632ef0030918000c200dd00007721007f
:1022a000008040001000be000001be00309280009f
:1022b00041928000800f5100818f59000900310048
:1022c00030918000c200dd000077210000804000d6
:1022d0001000be00309288004192880026d2bf00d4
:1022e00062f2b7002632ec0031918000e28f50009c
:1022f000e8ff3a006312a9000000060020c4b30002
:102300005c52e30021003a005d52e2001d003a00f9
:102310002632ef0031918000e18f500009003e002d
:1023200030918000c200dd00007721000081400074
:10233000f0ff2f00f1ff2f000089be002632ec00d5
:10234000f4ff39002a32ef006312a80014cea9006e
:10235000042ea900000028006091880000002800d9
:102360007091880000002800809188006d72ef0055
:1023700080938000c091880080938000d091880075
:1023800001003700042ea80014003700b0c7b300c6
:102390005c52e30011003a0014cea90000002800ae
:1023a00060918800000028007091880000002800db
:1023b0008091880070b7ef0072b7ef0074b7ef003c
:1023c00076b7ef002a32ef006d72ef008093800045
:1023d000c091880080938000d09188005cf2ef006b
:1023e0000000060070b6ef00101a2f0090b38800ae
:1023f00010412e00a0b3880040742d00b0b38800b7
:10240000f0b22c00c0b3880070fc2b00d0b3880061
:1024100030502b00e0b38800a0ad2a00f0b3880054
:1024200030142a0000b488006083290010b48800aa
:10243000b0fa280020b48800a079280030b48800c1
:10244000c00020003091880031918000f78f50004b
:102450000e003e00c00020002612b50000067800e5
:102460000c0646000067210060007e004100de008f
:10247000329180004111dd0001672100010141001e
:10248000000978002632ec00efff390080012000bf
:10249000309188003191800030022000808f500000
:1024a0000e003e00800120002612b50000067800d4
:1024b0000c0646000067210060007e004200de003e
:1024c000329180004111dd000167210001014100ce
:1024d000000978002632ec00eeff390040022000af
:1024e0003091880031918000f0022000808f5000f0
:1024f0000e003e00400220002612b50000067800c3
:102500000c0646000067210060007e004300de00ec
:10251000329180004111dd0001672100010141007d
:10252000000978002632ec00eeff3900000320009d
:102530003091880031918000b0032000808f5000de
:102540000e003e00000320002612b50000067800b1
:102550000c0646000067210060007e004400de009b
:10256000329180004111dd0001672100010141002d
:10257000000978002632ec00eeff3900c00320008d
:10258000309188003191800070042000808f5000cd
:102590000e003e00c00320002612b50000067800a1
:1025a0000c0646000067210060007e004500de004a
:1025b000329180004111dd000167210001014100dd
:1025c000000978002632ec00eeff3900800420007c
:1025d000309188003191800030052000808f5000bc
:1025e0000e003e00800420002612b5000006780090
:1025f0000c0646000067210060007e004600de00f9
:10260000329180004111dd0001672100010141008c
:10261000000978002632ec00eeff3900007a210034
:10262000c0b88800f0732100d0b88800f06d210098
:10263000e0b8880000682100f0b8880040622100fe
:1026400000b98800805c210010b98800e0562100a4
:1026500020b988006051210030b98800f04b21007a
:1026600040b988009046210050b9880050412100af
:1026700060b98800203c210070b988001037210023
:1026800080b988001032210090b98800202d2100e7
:10269000a0b9880040282100b0b98800802321001b
:1026a000c0b98800d01e2100d0b98800301a21009e
:1026b000e0b98800a0152100f0b9880020112100a0
:1026c00000ba8800c00c210010ba880070082100f0
:1026d00020ba88002004210030ba8800f0ff2000d2
:1026e00040ba8800d0fb200050ba8800c0f7200014
:1026f00060ba8800d0f3200070ba8800e0ef2000b4
:1027000080ba880000ec200090ba880030e82000f1
:10271000a0ba880070e42000b0ba8800c0e02000b1
:10272000c0ba880020dd2000d0ba880090d92000ef
:10273000e0ba880010d62000f0ba8800a0d22000ad
:1027400000bb880040cf200010bb8800e0cb2000f9
:1027500020bb8800a0c8200030bb880060c52000d6
:1027600040bb880030c2200050bb880010bf200052
:1027700060bb880000bc200070bb88000000060021
:1027800070b5ef00a0c7250090ab880050982500d9
:10279000a0ab880040812500b0ab8800906a25007e
:1027a000c0ab880030542500d0ab8800303e2500f7
:1027b000e0ab880090282500f0ab8800501325007e
:1027c00000ac880060fe240010ac8800c0e9240042
:1027d00020ac880080d5240030ac880090c1240053
:1027e00040ac8800f0ad240050ac8800a09a2400d2
:1027f00060ac8800a087240070ac8800f0742400ce
:1028000080ac88009062240090ac88008050240046
:10281000a0ac8800b03e2400b0ac8800302d24006d
:10282000c0ac8800f01b2400d0ac8800000b240052
:10283000e0ac880050fa2300f0ac8800e0e9230007
:1028400000ad8800c0d9230010ad8800e0c9230086
:1028500020ad880040ba230030ad8800e0aa2300f4
:1028600040ad8800c09b230050ad8800e08c230061
:1028700060ad8800307e230070ad8800d06f2300eb
:1028800080ad8800a061230090ad8800b053230084
:10289000a0ad8800f0452300b0ad8800703823005b
:1028a000c0ad8800202b2300d0ad8800101e23006f
:1028b000e0ad880040112300f0ad880090042300b3
:1028c00000ae880020f8220010ae8800e0eb220065
:1028d00020ae8800d0df220030ae8800f0d3220086
:1028e00040ae880050c8220050ae8800d0bc220004
:1028f00060ae880080b1220070ae880070a6220011
:1029000080ae8800809b220090ae8800c09022009c
:10291000a0ae880020862200b0ae8800c07b2200d6
:10292000c0ae880080712200d0ae880060672200af
:10293000e0ae8800805d2200f0ae8800c053220027
:1029400000af8800204a220010af8800b04022006b
:1029500020af88006037220030af8800402e220070
:1029600040af88004025220050af8800601c220044
:1029700060af8800b013220070af8800200b2200e7
:1029800080af8800b002220090af880060fa21007a
:10299000a0af880040f22100b0af880030ea2100eb
:1029a000c0af880050e22100d0af880090da21004b
:1029b000e0af8800e0d22100f0af880060cb2100ba
:1029c00000b08800f0c3210010b08800b0bc210026
:1029d00020b0880080b5210030b0880080ae210092
:1029e00040b0880090a7210050b08800b0a021001e
:1029f00060b08800009a210070b0880060932100c8
:102a000080b08800e08c210090b088008086210092
:102a1000a0b0880030802100b0b08800007a21008a
:102a2000c0b08800f0732100d0b08800f06d2100a4
:102a3000e0b0880000682100f0b08800406221000a
:102a400000b18800805c210010b18800e0562100b0
:102a500020b188006051210030b18800f04b210086
:102a600040b188009046210050b1880050412100bb
:102a700060b18800203c210070b18800103721002f
:102a800080b188001032210090b18800202d2100f3
:102a9000a0b1880040282100b0b188008023210027
:102aa000c0b18800d01e2100d0b18800301a2100aa
:102ab000e0b18800a0152100f0b1880020112100ac
:102ac00000b28800c00c210010b2880070082100fc
:102ad00020b288002004210030b28800f0ff2000de
:102ae00040b28800d0fb200050b28800c0f7200020
:102af00060b28800d0f3200070b28800e0ef2000c0
:102b000080b2880000ec200090b2880030e82000fd
:102b1000a0b2880070e42000b0b28800c0e02000bd
:102b2000c0b2880020dd2000d0b2880090d92000fb
:102b3000e0b2880010d62000f0b28800a0d22000b9
:102b400000b3880040cf200010b38800e0cb200005
:102b500020b38800a0c8200030b3880060c52000e2
:102b600040b3880030c2200050b3880010bf20005e
:102b700060b3880000bc200070b38800000006002d
:102b800090dc230060928800b0fd20005092880005
:102b90002632ef0027f2bf0019003a00529280005f
:102ba0006392800030918000e0f7070066f707002d
:102bb0002cf6070070928800819288007292800043
:102bc000839280000000200001f8230000f7070036
:102bd0000001be0000c02f00f16724005af7070073
:102be000b3f70700329180004111dd000137210069
:102bf00001014100000978002632ec00e5ff3900b0
:102c00000000060040122000709b8800c0122000c7
:102c1000609b880060132000509b8800b013200048
:102c2000409b880000142000309b88005014200036
:102c3000209b8800b0142000109b88000015200005
:102c4000009b880060152000f09a8800b0152000d5
:102c5000e09a880010162000d09a88007016200094
:102c6000c09a8800d0162000b09a88003017200043
:102c7000a09a880090172000909a8800f0172000f2
:102c8000809a880050182000709a8800b0182000a0
:102c9000609a880020192000509a8800801920002e
:102ca000409a8800f0192000309a8800601a2000ad
:102cb000209a8800d01a2000109a8800401b20001b
:102cc000009a8800b01b2000f0998800201c20008a
:102cd000e0998800a01c2000d0998800101d2000d9
:102ce000c0998800901d2000b0998800101e200017
:102cf000a0998800801e200090998800001f200065
:102d000080998800901f2000709988001020200072
:102d10006099880090202000509988002021200090
:102d200040998800a021200030998800302220009e
:102d300020998800c022200010998800502320008c
:102d400000998800f0232000f0988800802420005b
:102d5000e098880020252000d0988800b025200029
:102d6000c098880050262000b0988800f0262000e7
:102d7000a098880090272000909888004028200084
:102d800080988800e0282000709888009029200012
:102d900060988800402a200050988800f02a20007f
:102da00040988800a02b200030988800602c2000dc
:102db00020988800102d200010988800d02d200029
:102dc00000988800902e2000f0978800502f200057
:102dd000e097880020302000d0978800e030200065
:102de000c0978800b0312000b09788008032200062
:102df000a09788005033200090978800303420003e
:102e0000809788001035200070978800e0352000fa
:102e100060978800d036200050978800b037200097
:102e20004097880090382000309788008039200033
:102e300020978800703a200010978800703b20008f
:102e400000978800603c2000f0968800603d2000dc
:102e5000e0968800603e2000d0968800703f2000f9
:102e6000c096880070402000b09688008041200005
:102e7000a09688009042200090968800b0432000e1
:102e800080968800c044200070968800e0452000ad
:102e90006096880010472000509688003048200037
:102ea000409688006049200030968800a04a2000a3
:102eb00020968800d04b200010968800104d2000ee
:102ec00000968800504e2000f0958800a04f20000a
:102ed000e0958800f0502000d095880040522000f6
:102ee000c095880090532000b0958800f0542000d1
:102ef000a09588005056200090958800c05720006b
:102f0000809588003059200070958800a05a2000d4
:102f100060958800205c200050958800a05d20000e
:102f200040958800305f200030958800c060200008
:102f3000209588005062200010958800f0632000e2
:102f40000095880090652000f0948800406720007c
:102f5000e0948800f0682000d0948800a06a2000e7
:102f6000c0948800606c2000b0948800306e20000f
:102f7000a0948800f06f200090948800d071200009
:102f800080948800b07320007094880090752000b1
:102f90006094880080772000509488007079200029
:102fa00040948800707b200030948800707d200061
:102fb00020948800807f200010948800a081200049
:102fc00000948800c0832000f0938800e0852000f2
:102fd000e093880010882000d0938800508a200059
:102fe000c0938800908c2000b0938800e08e200071
:102ff000a093880030912000909388009093200047
:103000008093880080938000409188002632ef00f2
:1030100031918000f0072000808f500010003e00aa
:1030200032918000020141000027210060007900f8
:103030008000780040918000808f500006003e00a4
:103040002832ed004291800030918000818721007c
:1030500080707900f2ff37002632ec00ecff390077
:0c3060002832ef0000000600ffff3700e0
:020000040000fa
:10306c001a1200000c000000800000002612000064
:10307c0018000000800000003e1200001400000048
:10308c0080000000521200001e00000080000000b2
:10309c007012000000050000800000007017000096
:1030ac0008000000800000007817000000110000ec
:0830bc0080000000000000008c
:00000001FF
